:100000000C94AC010C94C9010C94C9010C94C90165
:100010000C94C9010C94C9010C94C9010C94C90138
:100020000C94C9010C94C9010C94C9010C94C90128
:100030000C94C9010C94C9010C94C9010C94C90118
:100040000C94C9010C94C9010C94C9010C94C90108
:100050000C94C9010C94C9010C94C9010C94C901F8
:100060000C94C9010C94C901AE2000B0C800104026
:10007000813FA1A6A83FA4D300D5F0D922DA12DB94
:10008000208D140000000000000000002F00000080
:10009000000700070000147F147F1400242A7F2A21
:1000A00012006264081323003649552250000005EF
:1000B00003000000001C224100000041221C00003F
:1000C00014083E08140008083E0808000000A0605C
:1000D0000000080808080800006060000000201008
:1000E000080402003E5149453E0000427F400000A6
:1000F0004261514946002141454B31001814127F9D
:1001000010002745454539003C4A494930000171F6
:1001100009050300364949493600064949291E00A8
:100120000036360000000056360000000814224158
:1001300000001414141414000041221408000201D9
:1001400051090600324959513E007C1211127C00BF
:100150007F49494936003E41414122007F414122C9
:100160001C007F49494941007F09090901003E41BE
:1001700049497A007F0808087F0000417F4100005C
:100180002040413F01007F08142241007F40404051
:1001900040007F020C027F007F0408107F003E4178
:1001A00041413E007F09090906003E4151215E00A0
:1001B0007F091929460046494949310001017F015B
:1001C00001003F4040403F001F2040201F003F40B3
:1001D00038403F00631408146300070870080700E4
:1001E000615149454300007F41410000552A552A8D
:1001F00055000041417F000004020102040040401C
:100200004040400000010204000020545454780093
:100210007F4844443800384444442000384444482B
:100220007F00385454541800087E0901020018A4B5
:10023000A4A47C007F080404780000447D400000F2
:100240004080847D00007F102844000000417F40F2
:1002500000007C04180478007C080404780038440A
:1002600044443800FC242424180018242418FC00DA
:100270007C0804040800485454542000043F4440BF
:1002800020003C4040207C001C2040201C003C40C2
:1002900030403C004428102844001CA0A0A07C0052
:1002A0004464544C4400000877410000000063009F
:1002B00000000041770800000804080804003A40E4
:1002C00040207A003D4040403D0021545454790084
:1002D0007D1211127D003944444439003D424242AE
:1002E0003D000205020000007E01495573007C10AC
:1002F00010081CFC5FDC60E461C462F663D664B085
:1003000065DF66B567FFFF32393034313931373553
:100310003400200032003500370031003900310050
:1003200034003000390032202020202020202020DE
:1003300000B53D2521003236303431393136333085
:1003400000436F6E7472617374464600466C61734D
:10035000682020313233000011241FBECFEFD8E0D7
:10036000DEBFCDBF11E0A0E0B1E0EEE3FDE002C0F2
:1003700005900D92AC30B107D9F711E0ACE0B1E0D7
:1003800001C01D92A031B107E1F70E94F8040C945E
:100390009D060C9400001092B9008CE58093B80083
:1003A00084E08093BC000895982F84EA8093BC0079
:1003B00020E931E007C02150304021F480910E0146
:1003C000816015C08091BC0087FD03C021153105F7
:1003D00091F79093BB0084E88093BC0020E931E062
:1003E00009C02150304031F480910E018260809329
:1003F0000E0108958091BC0087FD03C021153105D1
:1004000081F7089584E98093BC0008958093BB0030
:1004100084E88093BC0020E931E009C021503040DD
:1004200031F480910E01846080930E0108958091D3
:10043000BC0087FD03C02115310581F7089584ECC8
:100440008093BC0020E931E00AC02150304039F4EB
:1004500080910E01886080930E0180E00895809164
:10046000BC0087FD03C02115310579F78091BB00E1
:10047000089584E88093BC0020E931E00AC021504F
:10048000304039F480910E01806180930E0180E04C
:1004900008958091BC0087FD03C02115310579F7CF
:1004A0008091BB000895FF920F931F93CF93DF932A
:1004B000182F092FF62E88E70E94D40180E00E94B1
:1004C0000602212F302FC901EC0110E004C08991F0
:1004D0000E9406021F5F1F15D0F384E98093BC00C1
:1004E000DF91CF911F910F91FF900895EF92FF92AE
:1004F0000F931F93CF93DF937C018B0188E70E94BA
:10050000D40180E40E940602C0E0D0E007C0F701F9
:10051000EC0FFD1F80810E9406022196C017D107B3
:10052000B0F384E98093BC00DF91CF911F910F91CC
:10053000FF90EF900895DF93CF9300D000D0CDB718
:10054000DEB7982F8631B0F46830A0F486E0989F2B
:10055000C001112480930C0160930D0160556983E3
:1005600021E22A838B838FE78C83CE01019664E09E
:100570000E9453020F900F900F900F90CF91DF9138
:10058000089580E060E00E949B0208951F93DF932E
:10059000CF930F92CDB7DEB7182F88E70E94D40112
:1005A000113011F086EA01C087EA8983CE010196F5
:1005B00061E00E9453020F90CF91DF911F91089547
:1005C0001F93DF93CF930F92CDB7DEB7182F88E735
:1005D0000E94D401113011F08FEA01C08EEA8983A4
:1005E000CE01019661E00E9453020F90CF91DF91FE
:1005F0001F910895DF93CF9300D0CDB7DEB791E878
:1006000099838A83CE01019662E00E9453020F9083
:100610000F90CF91DF9108956F927F929F92AF924A
:10062000BF92CF92DF92EF92FF920F931F93DF93CF
:10063000CF93CDB7DEB760970FB6F894DEBF0FBE8D
:10064000CDBF8930D9F08A3020F4883009F041C01C
:1006500005C08A3069F18D30E1F535C010910B018C
:1006600080910C01811B60910D010E949B0280E230
:100670000E940C0380910C01811B26C060910C012B
:1006800080910B01482F50E0440F551F440F551F18
:100690009A01260F311D88279927841B950B4596B3
:1006A0002817390718F4862F840F0EC085E10CC077
:1006B00060910D01673008F0F8C080910B01680F60
:1006C00080910C0103C080E060910D010E949B02AB
:1006D000ECC090900C0129E7291508F4E6C080329F
:1006E00008F4E3C0182F1052E4EFF2E0E4911E1773
:1006F000D8F020E0412F50E00CC08D509D4FFC0100
:10070000849190E080978417950711F4132F0CC003
:100710002F5F822F90E0880F991FFC01EC50FD4F56
:1007200034913F3F51F7C1C080910B01823009F0F5
:100730009FC045E0A42EB12CAC0EBD1E86E0189FD4
:10074000F0011124ED57FF4F650101E010E031E1A8
:10075000E32EF12CEC0EFD1ED6011D921C9284910D
:1007600040E050E061E070E0682E7724C301042E81
:1007700002C0959587950A94E2F780FF1BC0CA01D5
:10078000880F991F980102C0220F331F8A95E2F744
:10079000C901D6012D913C911197822B932B980181
:1007A000062E02C0220F331F0A94E2F7822B932BEE
:1007B0008D939C934F5F5F4F6E5F7F4F4830510525
:1007C000A9F622E030E0C20ED31E3196CE14DF042B
:1007D00009F0C2CF88E70E94D40180E40E9406029B
:1007E0007501D7011C91812F0E940602812F0E9462
:1007F0000602E2E0F0E0EE0EFF1EEC14FD0489F7C5
:1008000084E98093BC0000910D010F540983015BC2
:1008100081E28A839B828FE78C83CE01019664E01C
:100820000E94530288E70E94D40180E40E940602DD
:10083000D50111961C91812F0E940602812F0E94E2
:100840000602E2E0F0E0AE0EBF1EAC14BD0481F77C
:1008500084E98093BC0000550983192D145F1B8324
:10086000CE01019664E00E94530210930C011DC05A
:1008700088E70E94D40180E40E94060286E0189F67
:10088000800111240D571F4FFF24F80184910E940D
:100890000602F3940F5F1F4FF6E0FF16B1F784E9ED
:1008A0008093BC009F0E90920C0160960FB6F89456
:1008B000DEBF0FBECDBFCF91DF911F910F91FF9093
:1008C000EF90DF90CF90BF90AF909F907F906F9010
:1008D000089580930B010895CF93DF93EC0103C03B
:1008E00021960E940C0388818823D1F7DF91CF9154
:1008F0000895CF93DF93EC0102C00E940C03FE0128
:10090000219684918823C9F7DF91CF91089520EA39
:100910003FE004C0F9013197F1F701970097D1F753
:100920000895FF920F931F93DF93CF93CDB7DEB758
:10093000C058D0400FB6F894DEBF0FBECDBFFE0149
:10094000319680E8DF011D928A95E9F710E0FE2ECE
:100950000F2F80E0612F0E949B028F2D902F60E867
:1009600070E00E9476021F5F183099F70E94C10262
:10097000C058DF4F0FB6F894DEBF0FBECDBFCF918A
:10098000DF911F910F91FF900895DF93CF93CDB723
:10099000DEB76C970FB6F894DEBF0FBECDBF482F01
:1009A0001092B9008CE58093B80084E08093BC007D
:1009B00020E030E0CE010196F901E859FF4FE491C3
:1009C000DC01A20FB31FEC932F5F3F4F2B3131059A
:1009D00099F74C8F6CE10E9453020E9491046C962F
:1009E0000FB6F894DEBF0FBECDBFCF91DF91089553
:1009F000CF92DF92EF92FF920F931F93CF93DF93EB
:100A00008FEA0E94C5048FEF0E94FA0281E0809372
:100A10000B0180930F0112E0F12E03E0C0EADFE04A
:100A2000B6E0EB2EA5E0CA2EF7E0DF2E80910F0195
:100A300080910F0180E060E00E949B0280E091E0E5
:100A40000E946C0480910F0160910F0180E00E9470
:100A50009B028CE493E00E94790480910F016091E5
:100A60000F0170E0660F771F80E00E949B0281E417
:100A700093E00E94790480910F0160910F01609FC3
:100A8000B001112480E00E949B0286E393E00E9463
:100A9000790488E893E1FE013197F1F70197D9F7DE
:100AA00081E00E94C60280910F0160910F01609F5A
:100AB000B00111248E9D802D11240E949B0281E3A0
:100AC00093E00E94790488E893E1FE013197F1F701
:100AD0000197D9F780E00E94C60280910F016091D2
:100AE0000F01609FB001112480E00E949B0286E20A
:100AF00093E00E94790488EC90E0FE013197F1F7D1
:100B00000197D9F780910F0160910F01609FB001AB
:100B100011240E949B0284E293E00E94790488ECF5
:100B200090E0FE013197F1F70197D9F780910F011D
:100B300060910F01609FB0011124880F0E949B02F9
:100B400082E293E00E94790488EC90E0FE01319704
:100B5000F1F70197D9F780910F0160910F01609F24
:100B6000B0011124809F802D11240E949B0280E2FD
:100B700093E00E94790488EC90E0FE013197F1F750
:100B80000197D9F780910F0160910F01609FB0012B
:100B90001124880F880F0E949B028EE193E00E942F
:100BA000790488EC90E0FE013197F1F70197D9F7CD
:100BB00080910F0160910F01609FB00111248C9D05
:100BC000802D11240E949B028CE193E00E94790405
:100BD00088EC90E0FE013197F1F70197D9F7809109
:100BE0000F0160910F01609FB00111248E9D802D37
:100BF00011240E949B028AE193E00E94790488EC10
:100C000090E0FE013197F1F70197D9F780910F013C
:100C100060910F01609FB00111248D9D802D1124E2
:100C20000E949B0288E193E00E94790488EC90E0A6
:100C3000FE013197F1F70197D9F780910F0160918B
:100C40000F01609FB0011124880F880F880F0E9448
:100C50009B0286E193E00E94790488EC90E0FE011B
:100C60003197F1F70197D9F780910F0160910F014A
:100C7000609FB001112499E0899F802D11240E946A
:100C80009B0284E193E00E94790480ED97E0FE01ED
:100C90003197F1F70197D9F719E080910F01609131
:100CA0000F01609FB0011124189F802D11240E9414
:100CB0009B0282E193E00E94790488EC90E0FE01BF
:100CC0003197F1F70197D9F7115038F788E097E09D
:100CD000FE013197F1F70197D9F782E080930B017C
:100CE00080930F01FA9409F0A1CE80910F016091D9
:100CF0000F0183E0689FB001112480E00E949B02F5
:100D000087E093E00E94790488EB9BE020EA3FE0D3
:100D1000F9013197F1F70197D9F781E00E94C602F6
:100D200088E893E120EA3FE0F9013197F1F7019774
:0E0D3000D9F780E00E94C602FFCFF894FFCFF3
:0C0D3E00537472696E672052414D000131
:00000001FF
